:10000000FDC0000014C1000012C1000010C10000BA
:100010000EC100000CC100000AC1000008C10000B0
:1000200006C1000004C1000002C1000000C10000C0
:10003000FEC00000FCC00000FAC00000F8C00000D4
:10004000F6C00000F4C00000F2C00000F0C00000E4
:10005000EEC00000ECC00000EAC00000E8C00000F4
:10006000E6C00000E4C00000E2C00000E0C0000004
:10007000DEC00000DCC00000DAC00000D8C0000014
:10008000D6C00000D4C00000D2C00000D0C0000024
:10009000CEC00000CCC00000CAC00000C8C0000034
:1000A000C6C00000C4C00000C2C00000C0C0000044
:1000B000BEC00000BCC00000BAC00000B8C0000054
:1000C000B6C00000B4C00000B2C00000B0C0000064
:1000D000AEC00000ACC00000AAC00000A8C0000074
:1000E000A6C00000A4C00000A2C00000A0C0000084
:1000F0009EC000009CC000009AC0000098C0000094
:1001000096C0000094C0000092C0000090C00000A3
:100110008EC000008CC000008AC0000088C00000B3
:1001200086C0000084C0000082C0000080C00000C3
:100130007EC000007CC000007AC0000078C00000D3
:1001400076C0000074C0000072C0000070C00000E3
:100150006EC000006CC000006AC0000068C00000F3
:1001600066C0000064C0000062C0000060C0000003
:100170005EC000005CC000005AC0000058C0000013
:1001800056C0000054C0000052C0000050C0000023
:100190004EC000004CC000004AC0000048C0000033
:1001A00046C0000044C0000042C0000040C0000043
:1001B0003EC000003CC000003AC0000038C0000053
:1001C00036C0000034C0000032C0000030C0000063
:1001D0002EC000002CC000002AC0000028C0000073
:1001E00026C0000024C0000022C0000020C0000083
:1001F0001EC000001CC000001AC0000011241FBE59
:10020000CFEFCDBFDFE3DEBF00E00CBF10E2A0E028
:10021000B0E2E8E2F9E400E00BBF02C007900D9203
:10022000A230B107D9F70E94EA230C949224E8CEB9
:10023000FC0180E090E4808391839170DB018D93D9
:100240009C938181869580831182089544ED57E0C7
:1002500060E070E08091D10080FDFCCF82EE809361
:10026000D000000082E28093D0008AE38093CA012C
:100270004093C001BB27A72F962F852F8093C101E4
:100280001092C20180E090E4AA2797FDA095BA2FB2
:100290000197A109B109840F951FA61FB71F80936D
:1002A000C401492F5A2F6B2F77274093C501CD01E9
:1002B000AA27BB278093C60188ED84BF8091CB011C
:1002C00081608093CB018091CF0187FDFCCF80912D
:1002D000D10080FDFCCF4091D7006091D6002091E5
:1002E000D5003091D400862F90E0A0E0B0E07727D1
:1002F0006627942B632B1092D000722B08958F9257
:100300009F92AF92BF92CF92DF92EF92FF920F93A4
:100310001F93CF93DF932FEF3FEFFC0120833183B7
:10032000C0E0D0E46E01CD2CDD24C694E12CF12C8C
:100330004C155D056E057F0538F04C155D056E05A5
:100340007F0529F4D17005C0C0E0D2E002C0C0E052
:10035000D0E06A017B0139E0CC0CDD1CEE1CFF1CF7
:100360003A95D1F724ED37E0C20ED31EE11CF11C03
:100370008C01C80FD91F46015701C4018C199D0972
:100380000C171D0769F040E0C501B40162D0F80107
:1003900081938F01FFEF8F1A9F0AAF0ABF0AEDCF3B
:1003A000DF91CF911F910F91FF90EF90DF90CF9051
:1003B000BF90AF909F908F90089520E032E0215041
:1003C0003109FC01E20FF31F5081FB01E20FF31F23
:1003D0004081541729F0451748F481E090E00895D2
:1003E0002115310561F780E090E008958FEF9FEFD0
:1003F0000895BF92CF92DF921F93CF93DF93DC01DA
:10040000CB01142FE9013FB7F894E0E0FFE00F9231
:100410001F927DEF6FEF5FEF40E8D92EC82EBA2E06
:1004200020913C002F9321E020933C00212F1D2E92
:100430000C2E19950F9000923C001F900F902F3FAB
:10044000F9F33FBFDF91CF911F91DF90CF90BF9025
:100450000895CF92DF92EF92FF921F936C01EE24EA
:10046000FF24FB0110913B00C0923B004093CA0166
:10047000D895802D10933B001F91FF90EF90DF9057
:10048000CF9008958F929F92AF92BF92CF92DF92BA
:10049000EF92FF920F931F93CF93DF931F92CDB7ED
:1004A000DEB74A015B0139E0880C991CAA1CBB1C11
:1004B0003A95D1F78C01C12CD12C7601C701B60138
:1004C000680D791D8A1D9B1D422F2983C2DFF8010B
:1004D00081938F01FFEFCF1ADF0AEF0AFF0A29810C
:1004E000C11482E0D806E104F10441F780E092E013
:1004F0000F90DF91CF911F910F91FF90EF90DF90C0
:10050000CF90BF90AF909F908F900895AF92BF9281
:10051000CF92DF92EF92FF920F931F93CF93DF93CF
:100520001F92CDB7DEB75C016A017B0149E0CC0CBC
:10053000DD1CEE1CFF1C4A95D1F700E012E00150D3
:100540001109C701B601600F711F811D911D422F56
:1005500029837FDFF501E00FF11F90812981981732
:1005600029F0981748F48FEF9FEF08C00115110587
:1005700031F780E090E002C081E090E00F90DF91E1
:10058000CF911F910F91FF90EF90DF90CF90BF9090
:10059000AF90089520E076CF20E0B8CFE8E0FFE00C
:1005A0007DEF6FEF5FEF40E820913C002F9321E05B
:1005B00020933C0019950F9000923C00822F80956B
:1005C0000895EAE0FFE020913C002F9321E0209382
:1005D0003C0019950F9000923C002F3F19F4BB2767
:1005E000A0E207C0203019F4BFEFAFEF02C0BB2775
:1005F000A22FCD010895EEE0FFE020913C002F9363
:1006000021E020933C00282F19950F9000923C0088
:10061000822F08954F925F926F927F928F929F9256
:10062000AF92BF92CF92DF92EF92FF920F931F9300
:10063000CF93DF93EC014B0169017A0169E0CC0CA7
:10064000DD1CEE1CFF1C6A95D1F716E21093CA015F
:100650002091CB01216018ED109334002093CB0141
:100660001091CF011078E1F726013701A12CB12CB0
:10067000F401EA0DFB1D218130E0322F2227808119
:10068000282B10913C008A818F778CBFE881F981FB
:1006900043E2C301B201199510933C0082E0A80E19
:1006A000B11C82E0480E511C611C711CA11482E037
:1006B000B806F1F610913C008A818F778CBFE881F3
:1006C000F98120E030E0402FC701B6011995109361
:1006D0003C0080E092E0DF91CF911F910F91FF905D
:1006E000EF90DF90CF90BF90AF909F908F907F90D2
:1006F0006F905F904F9008958F929F92AF92BF92AC
:10070000CF92DF92EF920F93CF93DF936C01EB01C7
:1007100049015A01202FB501A401CE01F7DE892B32
:1007200039F00E2DA5019401BE01C60173DF02C090
:1007300080E092E0DF91CF910F91EF90DF90CF902A
:10074000BF90AF909F908F9008950F93CF93DF93BA
:1007500000D0CDB7DEB7E0E029EF31E029833A835E
:10076000EB830FE29A01AB01BC01CE01019652DF8F
:100770002396CDBFDEBFDF91CF910F910895CF9229
:10078000DF92EF92FF92CF93DF93EC016A017B013E
:1007900003DF892B51F0B701A601CE01DF91CF9184
:1007A000FF90EF90DF90CF90D0CF80E092E0DF918C
:1007B000CF91FF90EF90DF90CF90089580E01BDF06
:1007C0008A3531F48FEF17DF8A3511F480E813DFB3
:1007D0008FEF089580E180935500809150008061F3
:1007E000809350008091510084FFFCCF2FB7F89484
:1007F00034E088ED90E0A0E4B0E01BBEFD0184BFD2
:1008000030832FBF8FE39FE10197F1F700C0000015
:1008100080914000809150008260809350008091D0
:10082000510081FFFCCF8091560084608093560078
:1008300080E8809365008BEB8093660082E0809374
:10084000CA01EDE1F0E0E491E0936200ECE1F0E058
:10085000E491E09363001092CA0181E0809360000C
:1008600088ED84BF87E48093A20098D00F94AB0AF0
:100870004AD2811101C0FFCF45C20895089580E09A
:1008800090E20D947E0B80E090E20D944E0B80C2BE
:10089000292F33272230310539F02330310549F033
:1008A00021303105B9F01BC020E230E06CE970E284
:1008B0001AC099278330910590F4FC01EE0FFF1FB9
:1008C000E253FF4D60817181FC01EC52FF4D2081AC
:1008D00030E009C022E130E06CEB70E204C020E0BF
:1008E00030E060E070E0FA0160837183C90108952F
:1008F0000D940701CF92DF92EF92FF92CF93C091B8
:10090000B70688E18093B7068FE193E00197F1F78E
:1009100000C000008091A80687FF15C0C12CD12C13
:10092000760140E0C701B6010F9494018F3F71F446
:100930009FEFC91AD90AE90AF90AC11482E0D80658
:10094000E104F10471F70D9407010EC0C093B706DE
:10095000F0E4E0E0F0933E00E0933D0010923C00B4
:10096000FF27EE271995EFCFCF91FF90EF90DF9003
:10097000CF900895803829F08F3F21F0811104C075
:1009800001C0B6DF8AE508958FEF08958F93822F17
:100990002F91F0DF2F93282F8F91089515D380E0AA
:1009A00090E008959ED380E090E008952F923F92CA
:1009B0004F925F926F927F928F929F92AF92BF926F
:1009C000CF92DF92EF92FF920F931F93CF93DF931B
:1009D000CDB7DEB7C450D240CDBFDEBF5C01142F0F
:1009E000052FD62EC72E79010F94400A8111BAC067
:1009F000412F502F6D2D7C2D212C92E0392ECC24AF
:100A0000C394D12CCC0EDD1E4E018FEF881A8DEFD2
:100A1000980A94C0F601C10111920197E9F7860185
:100A20008091462190914721FC01EF5BFF4F20818F
:100A3000FC01E05CFF4F8081281718F4612C712CB9
:100A40002FC0CF5FDD4F4883C150D240CE5FDD4F16
:100A50005883C250D240CD5FDD4F6883C350D2402F
:100A6000CC5FDD4F7883C450D2400F9493080F942D
:100A7000400ACF5FDD4F4881C150D240CE5FDD4F8D
:100A80005881C250D240CD5FDD4F6881C350D24003
:100A9000CC5FDD4F7881C450D240882379F262C0A8
:100AA000CF5FDD4F4883C150D240CE5FDD4F5883CA
:100AB000C250D240CD5FDD4F6883C350D240CC5F7F
:100AC000DD4F7883C450D2400F94A208F801E60DA0
:100AD000F71D80839FEF691A790ACF5FDD4F488148
:100AE000C150D240CE5FDD4F5881C250D240CD5F61
:100AF000DD4F6881C350D240CC5FDD4F7881C45058
:100B0000D240E0E16E16710459F6F50180AD811115
:100B100029C0005F1F4F0815190509F081CF412C2E
:100B2000512C32014394440E551E661E771EC60199
:100B3000AFD3F1E0EF1AF108B301A201E114F1041F
:100B400009F068CF8091462190914721FC01EF5B2D
:100B5000FF4F2081FC01E05CFF4F8081281710F0DF
:100B60000F949308CC5FDD4FCDBFDEBFDF91CF91F7
:100B70001F910F91FF90EF90DF90CF90BF90AF90BB
:100B80009F908F907F906F905F904F903F902F90AD
:100B900008952F923F924F925F926F927F928F9221
:100BA0009F92AF92BF92CF92DF92EF92FF920F93FC
:100BB0001F93CF93DF93CDB7DEB7C450D240CDBFE4
:100BC000DEBF5C017901CF5FDD4F4883C150D24069
:100BD000CE5FDD4F5883C250D240CD5FDD4F68837A
:100BE000C350D240CC5FDD4F7883C450D2400F94C5
:100BF000400ACF5FDD4F4881C150D240CE5FDD4F0C
:100C00005881C250D240CD5FDD4F6881C350D24081
:100C1000CC5FDD4F7881C450D24081115CC01A0195
:100C20002B01CC24C394D12CCC0EDD1E40C0B201CC
:100C3000A101C601D9D24C0186012BC08091462169
:100C400090914721FC01EF5BFF4F2081FC01E05CAC
:100C5000FF4F8081281718F4612C712C07C00F9466
:100C60007A080F94400A8823B9F335C0F801E60DDD
:100C7000F71D80810F94B1088FEF681A780AE0E1C0
:100C80006E16710499F7F50180AD005F1F4F811159
:100C900022C0C8018C199D098815990578F2FFEFCB
:100CA0002F1A3F0A4F0A5F0A81E0E81AF108E1149F
:100CB000F10409F0BCCF8091462190914721FC01BD
:100CC000EF5BFF4F2081FC01E05CFF4F8081281724
:100CD00010F00F947A08CC5FDD4FCDBFDEBFDF91FF
:100CE000CF911F910F91FF90EF90DF90CF90BF9029
:100CF000AF909F908F907F906F905F904F903F90BC
:100D00002F900895089581E008950F931F93CF9336
:100D1000DF93EC01862F48A15F8D6E8D7D8D0BA139
:100D20001AA14F3191E059076105710568F0809172
:100D30003C20807F856080933C2081E28093462028
:100D40001092472080E01FC09801882319F0CE013F
:100D500020DF02C0CE012ADEC801A0E0B0E029E019
:100D6000880F991FAA1FBB1F2A95D1F74C895D894F
:100D70006E897F89481B590B6A0B7B0B4C8B5D8BF3
:100D80006E8B7F8B81E0DF91CF911F910F91089542
:100D9000CF92DF92EF92FF920F931F93CF93DF9347
:100DA000CDB7DEB72897CDBFDEBF8C01FC01838DA8
:100DB0008D3109F4A3C088F4823109F138F4882315
:100DC00009F4D8C0833009F0DBC045C08A3109F48A
:100DD000B5C08B3109F0D4C0CDC0883209F4AAC0A7
:100DE00038F48E3109F4C6C0853209F0C9C05BC041
:100DF0008A3209F49DC08F3209F0C2C0BBC0F8012D
:100E0000E78CF68C848D837009F07CC0858D811110
:100E100079C06701F5E2EF16F10418F044E2C42E40
:100E2000D12C40E050E0B60187ED90E20F9401072D
:100E300060E070E0C7018C199D090F94B6060F940D
:100E40007A08F80184899589A689B7898C199D0942
:100E5000A109B10923C0F801E78CFE2CF2E1FE15CF
:100E600010F432E1F32E40E050E06F2D70E08AE3A1
:100E700090E20F9401078E2D90E060E070E08F19F2
:100E800091090F94B6060F947A08F8018489958920
:100E9000A689B7898F199109A109B109848B958B0E
:100EA000A68BB78B79C08EE191E0A0E0B0E08D8396
:100EB0009E83AF83B88780E092E0A0E0B0E08983B2
:100EC0009A83AB83BC8340E050E064E070E0CE01E5
:100ED00005960F94540740E050E064E070E0CE01C6
:100EE00001960F9454070F947A08F8018489958924
:100EF000A689B7890897A109B109D0CFF801848DD7
:100F000082FD08C080913C20807F856080933C20DA
:100F100084E23DC0F8DE81112DC080913C20807FAD
:100F2000846080933C2010924620109247203FC05E
:100F300060E001C061E0C801E8DE2CC080E00F94F1
:100F4000B10880E00F94B10880E00F94B10880E010
:100F50000F94B1080F947A08F8014489558966897D
:100F600077894450510961097109448B558B668B0F
:100F7000778B12C0F801148A158A168A178A0CC05A
:100F800080913C20807F856080933C2080E280932C
:100F90004620CBCF882359F080913C20807F8093DE
:100FA0003C20109246201092472081E001C080E052
:100FB0002896CDBFDEBFDF91CF911F910F91FF909B
:100FC000EF90DF90CF900895CF92DF92EF92FF9253
:100FD0000F931F9372D1C1D1E9D2E6D40F9440048C
:100FE0000F944E040F9480040F94FC040F94040596
:100FF0000F941F0503D583E0C82ED12CE12CF12CD2
:1010000000E018E020E030E040E263E071E28BEFC6
:1010100090E24DD497E0C92ED12CE12CF12C00E0C8
:1010200012E020E030E040E263E071E286E091E22D
:101030003ED429E0C22ED12CE12CF12C00E010EEA0
:1010400021E030E040E263E071E28EE091E22FD4F3
:1010500039EFC32ED12CE12CF12C00E010E420E07C
:1010600030E041E263E071E286E191E220D449E1BF
:10107000C42EDD24D394E12CF12C0FE310E020E00A
:1010800030E041E263E071E28EE191E210D45BE195
:10109000C52EDD24D394E12CF12C00E410E020E0F7
:1010A00030E041E263E071E286E291E200D46DE17A
:1010B000C62EDD24D394E12CF12C02EA10E020E0CE
:1010C00030E041E266E371E28EE291E2F0D39BD23E
:1010D00080E090E01F910F91FF90EF90DF90CF9014
:1010E00008958FD40F9422050F9407050F94FF04E1
:1010F0000F948D040F9451040F944B0462D47ED24C
:101100002FD1DED080E090E008954F3121E05207EA
:101110006105710508F05FC04D3121E0520761059E
:10112000710528F04D515140610971096DC44B3171
:1011300021E052076105710530F04B5151406109C2
:1011400071090D942505493121E0520761057105AA
:1011500030F049515140610971090D940A05493F28
:1011600051056105710508F005C04930510561055B
:10117000710530F049505109610971090D9402055A
:10118000473051056105710530F04750510961093B
:1011900071090D949004433051056105710530F0DB
:1011A00043505109610971090D94540442305105AD
:1011B0006105710521F440E050E0BA0105C4452BFA
:1011C000462B472B21F040E050E0BA0114C340E029
:1011D00050E0BA015BC140E052E06FEF70E00F9465
:1011E000BE0C80E092E00895CF93DF93EC01CB0139
:1011F000BA010F946703AB01BC01CE01DF91CF911F
:1012000084CF4F3121E052076105710508F03DC0E0
:101210004B3121E0520761057105B8F5493F510591
:101220006105710590F5493051056105710530F092
:1012300049505109610971090D9403054730510561
:101240006105710530F047505109610971090D942C
:10125000B604433051056105710530F04350510922
:10126000610971090D946A044230510561057105E7
:1012700021F440E050E0BA01B4C3452B462B472B84
:1012800021F040E050E0BA01C3C280E090E0089550
:10129000CF93DF93EC01CB01BA010F946703AB014D
:1012A000BC01CE01AEDFEC011816190614F40F9440
:1012B000FE02CE01DF91CF91089580E090E0089585
:1012C00080E090E008958F929F92AF92BF92EF924C
:1012D000FF920F931F93CF93DF938C0180E092E0F6
:1012E000F8019C01119221503040E1F78BEEF8019A
:1012F00080838EEF818380E09EEFA1E0BB27E80131
:10130000C254DE4FBC01CD017B01F0E1EF0EF11CB8
:10131000812C912C54018394860E971EA81EB91E11
:1013200040E00F9494018993C501B401E814F904D5
:1013300079F7F801E250FE4F85E59AEA80839183C0
:1013400080E092E0DF91CF911F910F91FF90EF909D
:10135000BF90AF909F908F90089580E090E00895A7
:1013600080E090E0089583E008950F931F938B0130
:101370009C01369527951795079560FF02C00F5F72
:101380001F4FC8011F910F910895CF92DF92EF92E6
:10139000FF926B017C01E7DF90E0A0E0B0E0C816AF
:1013A000D906EA06FB0680F0A7019601281B390B37
:1013B0004A0B5B0BDA01C901B695A79597958795FE
:1013C0009C012E5F3F4F02C020E030E0C901FF903A
:1013D000EF90DF90CF900895CF92DF92EF92FF923F
:1013E0006B017C01C0DF482F50E060E070E0C41664
:1013F000D506E606F70628F09C2D981B892F8170EC
:1014000001C08C2DFF90EF90DF90CF900895CF9288
:10141000DF92EF92FF926B017C01A5DF90E0A0E0EC
:10142000B0E0C816D906EA06FB0628F0C701B601E7
:10143000D3DF91E0811190E0892FFF90EF90DF9052
:10144000CF900895CF92DF92EF92FF928230910574
:1014500098F06C01E12CF12C82E0C81AD108E10867
:1014600080E8F80ACC0CDD1CEE1CFF1C7CDFC80EEB
:10147000D11CE11CF11C03C0C12CD12C7601B6019A
:10148000C701FF90EF90DF90CF9008958F929F92C9
:10149000AF92BF92EF92FF920F931F93CF93DF9380
:1014A0008C0180E19EEFA1E0BB2720E032E0F80153
:1014B000A901119241505040E1F7E801BC01CD0172
:1014C0007B015EE3E50EF11C812C912C5401839489
:1014D000860E971EA81EB91E40E00F9494018993B2
:1014E000C501B401E814F90479F7F801E250FE4FA0
:1014F00085E59AEA8083918380E092E0DF91CF9145
:101500001F910F91FF90EF90BF90AF909F908F90A1
:101510000895969587959C01220F331F280F391F38
:10152000C90108951F93CF93DF93182FEB01F1DFCB
:10153000BE017F70FC013196DC01AA58BD4D10FF41
:1015400011C0EA58FD4D80818F70962F9295907F43
:10155000892B808354E0769567955A95E1F712962A
:101560006C9307C06C93EA58FD4D8081807F872B78
:101570008083DF91CF911F910895CF93C82FC9DF4A
:10158000FC01EA58FD4D8181C0FF08C082958F7033
:10159000228190E1299F9001112404C0382F3F70CF
:1015A00020E08081282BC901CF910895CF93DF934C
:1015B00080E092E0E6E7F2E2DF019C011D9221501B
:1015C0003040E1F768EF7FE080E090E0ABDF6FEF65
:1015D0007FE081E090E0A6DFC0E9D0E06FEF7FE040
:1015E000CE01A0DF2196C53531E0D307B9F70F94BE
:1015F0004E0380E090E0DF91CF9108950F945B035C
:1016000080E090E00895CF93DF93C2E0D0E0CE0178
:10161000B4DF892B21F467EF7FE0CE0183DF2196D1
:10162000C53581E0D80799F7DF91CF910895AF9242
:10163000BF92CF92DF92EF92FF920F931F93CF93BF
:10164000DF9300D01F92CDB7DEB76B017C012983F9
:101650003A834B835C83DBDE29813A814B815C8159
:10166000882369F1211531054105510541F1CA0170
:10167000B9017BDE5C01C701B60187DE7C0182E037
:10168000A816B10488F4C5018E0D9F1D6FEF7FE091
:10169000019748DF16C06901EFEFCE1ADE0AB601E6
:1016A000C90140DF960104C097018501015011096D
:1016B000C9018E199F098017910768F3E4CFE12CC7
:1016C000F12CC7012496CDBFDEBFDF91CF911F91D2
:1016D0000F91FF90EF90DF90CF90BF90AF90089563
:1016E0007F928F929F92AF92BF92CF92DF92EF92B2
:1016F000FF920F931F93CF93DF934B015C017A010D
:1017000044DE6C0130DE90E0A0E0B0E0881699067F
:10171000AA06BB0618F4C0E0D0E034C0712C872DB7
:1017200084D0EC01009749F18A8D9B8D00E010E098
:1017300020C0C816D906D1F416DEA5019401281BD5
:10174000310941095109CA01B90146DE20E030E002
:10175000000F111F221F331F080F111D211D311DE6
:10176000F70100831183228333830CC00F5F1F4F67
:1017700004DF883FFFE09F07E0F2739420E17212DC
:10178000CECFC9CFCE01DF91CF911F910F91FF90A6
:10179000EF90DF90CF90BF90AF909F908F907F9011
:1017A0000895CF92DF92EF92FF920F931F93CF9302
:1017B000DF937B01EC0100E010E00EC06801CE0C6D
:1017C000DF1CCE010F945E03B6010F94A0030F5FE0
:1017D0001F4FCE01D2DEEC01CE010297863F9F4023
:1017E00068F3C801DF91CF911F910F91FF90EF90A7
:1017F000DF90CF90089520E032E0E6E7F2E2DC01EE
:1018000001900D9221503040D9F780E092E0089588
:1018100020E032E0FC01A6E7B2E201900D922150F7
:101820003040D9F780E092E00895803160F490E292
:10183000899FF0011124EA56FA4D828D938D02970B
:1018400010F09F0102C020E030E0C9010895DF924E
:10185000EF92FF920F931F93CF93DF938C017B0145
:10186000D12C8D2DE2DFEC01009791F0BC01685F77
:101870007F4F43E050E0C7010F94C50C009741F43F
:1018800048E050E0BE01C8010F94C50C009731F04C
:10189000D39480E1D812E5CFC0E0D0E0CE01DF9153
:1018A000CF911F910F91FF90EF90DF9008954F928D
:1018B0005F926F927F929F92AF92BF92CF92DF9290
:1018C000EF92FF920F931F93CF93DF93EC015B0195
:1018D000942E2801390110E0812FA7DF892B41F4D4
:1018E000012F411451046104710439F40EEF4BC00F
:1018F0001F5F103189F70FEF46C0A301920189E005
:1019000056954795379527958A95D1F7D301C2010A
:101910009170AA27BB27892B8A2B8B2B21F02F5F55
:101920003F4F4F4F5F4FC701B60181DE82309105B7
:1019300048F120E21202B00111246A567A4D20E2E9
:10194000DB011D922A95E9F728E0FE01DB010190F9
:101950000D922A95E1F7F501208131814281DB0169
:1019600018962D933D934C931A971B969C921B9718
:101970005A968D939C935B97FB01448E558E668E91
:10198000778E01C00DEF802FDF91CF911F910F91C6
:10199000FF90EF90DF90CF90BF90AF909F907F909F
:1019A0006F905F904F90089580E092E0E6E9F5E255
:1019B000DF019C011D9221503040E1F780E090E072
:1019C000089580E090E0089520E032E0E6E9F5E255
:1019D000DC0101900D9221503040D9F780E092E077
:1019E000089520E032E0FC01A6E9B5E201900D92F5
:1019F00021503040D9F780E092E0089580E090E0F7
:101A0000089580E090E00895CF92DF92EF92FF92E8
:101A10000F931F93CF93DF930EE51EEF21E0332743
:101A2000FC01452B462B472B09F540E052E0DC0139
:101A3000BA011D9261507040E1F7EC01B801C90193
:101A400000E010E0C12CD12C7601C394C60ED71E45
:101A5000E81EF91E40E00F94940189930F5F1F4F19
:101A6000C701B601033A110569F708C080E092E0AA
:101A7000DF019C011D9221503040E1F780E092E0AF
:101A8000DF91CF911F910F91FF90EF90DF90CF905A
:101A900008950000000000000000000000000000A9
:101AA0000000000000000000000000000000000036
:101AB0000000000000000000000000000000000026
:101AC0000000000000000000000000000000000016
:101AD0000000000000000000000000000000000006
:1025D00000000000000002000404230001000000CD
:1025E0001E010000EBFE906D6B66732E6661740039
:1025F000020201000110001F01F8010001000100AA
:10260000000000001F010000800029785634124E9F
:102610004F204E414D45202020204641543132204C
:102620002020323031343037313154313530305A66
:1026300053425468697320697320616E206561722A
:102640006C792070726F746F7479706521205552A7
:102650004C20616E64206E616D65206D69676874E1
:10266000206E6F742062652066696E616C210D0AB0
:102670000D0A687474703A2F2F6D617472697873E3
:10268000746F726D2E636F6D2F6176722F6176722B
:10269000737469636B2F0D0A0D0A5374657068615A
:1026A0006E2042616572776F6C6620287374657066
:1026B00068616E406D617472697873746F726D2EAB
:1026C000636F6D292C20496C6D656E617520323009
:1026D00031340D0A0000000000000000000000007E
:1026E00000000000000000000000000000000000EA
:1026F00000000000000000000000000000000000DA
:1027000000000000000000000000000000000000C9
:1027100000000000000000000000000000000000B9
:1027200000000000000000000000000000000000A9
:102730000000000000000000000000000000000099
:102740000000000000000000000000000000000089
:102750000000000000000000000000000000000079
:102760000000000000000000000000000000000069
:102770000000000000000000000000000000000059
:102780000000000000000000000000000000000049
:102790000000000000000000000000000000000039
:1027A0000000000000000000000000000000000029
:1027B0000000000000000000000000000000000019
:1027C0000000000000000000000000000000000009
:1027D00000000000FDC0000024C1000022C1000074
:1027E00020C100001EC100001CC100001AC1000071
:1027F00018C1000016C1000014C1000012C1000081
:1028000010C100000EC100000CC1000015C1000085
:1028100008C1000006C1000004C1000002C10000A0
:1028200000C10000FEC00000FCC00000FAC00000B3
:10283000F8C00000F6C00000F4C00000F2C00000C4
:10284000F0C00000EEC00000ECC00000EAC00000D4
:10285000E8C00000E6C00000E4C00000E2C00000E4
:10286000E0C00000DEC00000DCC00000DAC00000F4
:10287000D8C00000D6C00000D4C00000D2C0000004
:10288000D0C00000CEC00000CCC00000CAC0000014
:10289000C8C00000C6C00000C4C00000C2C0000024
:1028A000C0C00000BEC00000BCC00000BAC0000034
:1028B000B8C00000B6C00000B4C00000B2C0000044
:1028C000B0C00000AEC00000ACC00000AAC0000054
:1028D000A8C00000A6C00000A4C00000A2C0000064
:1028E000A0C000009EC000009CC000009AC0000074
:1028F00098C0000096C0000094C0000092C0000084
:1029000090C000008EC000008CC000008AC0000093
:1029100088C0000086C0000084C0000082C00000A3
:1029200080C000007EC000007CC000007AC00000B3
:1029300078C0000076C0000074C0000072C00000C3
:1029400070C000006EC000006CC000006AC00000D3
:1029500068C0000066C0000064C0000062C00000E3
:1029600060C000005EC000005CC000005AC00000F3
:1029700058C0000056C0000054C0000052C0000003
:1029800050C000004EC000004CC000004AC0000013
:1029900048C0000046C0000044C0000042C0000023
:1029A00040C000003EC000003CC000003AC0000033
:1029B00038C0000036C0000034C0000032C0000043
:1029C00030C000002EC000000D94E10A2AC00000B3
:1029D00011241FBEDFE3CFEFDEBFCDBF1CBE0C94C2
:1029E00090F011241FBECFEFDFE3DEBFCDBF01E0CB
:1029F0000CBF11E2A0E0B0E2E6E5FAE102E00BBFB5
:102A000002C007900D92AA33B107D9F722E2AAE3D8
:102A1000B1E201C01D92A637B207E1F703D00D94D1
:102A2000290DD8CEF8940E9400F0789480E090E2CE
:102A30000F949B0B74D5FACF1F920F920FB60F9283
:102A400011240BB60F922F933F934F935F936F9385
:102A50007F938F939F93AF93BF93EF93FF930F94C5
:102A6000000F0F94400F0F949B0F0F948B0F0F9438
:102A7000940F0F94800FFF91EF91BF91AF919F91B1
:102A80008F917F916F915F914F913F912F910F9017
:102A90000BBE0F900FBE0F901F901895BF92CF9254
:102AA000DF921F93CF93DF93DC01CB01142FE90159
:102AB0003FB7F894E4E0FFE00F921F9270E060E00F
:102AC00050E040E0D92EC82EBA2E20913C002F9322
:102AD00021E020933C00212F1D2E0C2E19950F90E4
:102AE00000923C001F900F902F3FF9F33FBFDF9102
:102AF000CF911F91DF90CF90BF900895CF92DF923A
:102B0000EF92FF921F936C01EE24FF24FB011091C2
:102B10003B00C0923B004093CA01D895802D109392
:102B20003B001F91FF90EF90DF90CF9008958F9220
:102B30009F92AF92BF92CF92DF92EF92FF920F934C
:102B40001F93CF93DF931F92CDB7DEB74A015B018E
:102B500039E0880C991CAA1CBB1C3A95D1F78C0152
:102B6000C12CD12C7601C701B601680D791D8A1DD3
:102B70009B1D422F2983C2DFF80181938F01FFEF54
:102B8000CF1ADF0AEF0AFF0A2981C11482E0D806B2
:102B9000E104F10441F780E092E00F90DF91CF91E2
:102BA0001F910F91FF90EF90DF90CF90BF90AF906B
:102BB0009F908F900895AF92BF92CF92DF92EF9245
:102BC000FF920F931F93CF93DF931F92CDB7DEB782
:102BD0005C016A017B0149E0CC0CDD1CEE1CFF1C92
:102BE0004A95D1F700E012E001501109C701B60182
:102BF000600F711F811D911D422F29837FDFF50119
:102C0000E00FF11F90812981981729F0981748F457
:102C10002FEF3FEF08C00115110531F720E030E03C
:102C200002C021E030E0C9010F90DF91CF911F91E8
:102C30000F91FF90EF90DF90CF90BF90AF900895ED
:102C400020E075CF20E0B7CF4F925F926F927F92D6
:102C50008F929F92AF92BF92CF92DF92EF92FF92AC
:102C60000F931F93CF93DF935B0169017A0159E0C2
:102C7000CC0CDD1CEE1CFF1C5A95D1F716E210930C
:102C8000CA012091CB01216018ED109334002093EC
:102C9000CB011091CF011078E1F726013701812C8B
:102CA000912CF501E80DF91D8181D82F80E0C82F06
:102CB00080819E01282B43E2C301B201EFDE82E056
:102CC000880E911C82E0480E511C611C711C8114FD
:102CD00082E0980631F720E030E0402FC701B601CE
:102CE000DDDE80E092E0DF91CF911F910F91FF90A8
:102CF000EF90DF90CF90BF90AF909F908F907F909C
:102D00006F905F904F9008958F929F92AF92BF9275
:102D1000CF92DF92EF920F93CF93DF936C01EB0191
:102D200049015A01202FB501A401CE0144DF892BAE
:102D300041F00E2DA5019401BE01C60185DF9C0165
:102D400002C020E032E0C901DF91CF910F91EF90F6
:102D5000DF90CF90BF90AF909F908F9008950F938A
:102D6000CF93DF9300D0CDB7DEB7E1E024E631E0CA
:102D700029833A83EB830FE29A01AB01BC01CE01B8
:102D8000019662DF2396CDBFDEBFDF91CF910F9119
:102D90000895CF92DF92EF92FF92CF93DF93EC01F1
:102DA0006A017B014FDF892B51F0B701A601CE01EB
:102DB000DF91CF91FF90EF90DF90CF90D0CF80E068
:102DC00092E0DF91CF91FF90EF90DF90CF90089548
:102DD0000F931F93CF93DF9363E071E28BEF90E249
:102DE0000E943DF8EC01009769F063E070E080E03C
:102DF00090E00E94DBF5BC018A8D9B8D0E94E7F775
:102E0000EC0102C0C0E0D0E063E071E286E091E254
:102E10000E943DF88C01009771F067E070E080E05F
:102E200090E00E94DBF5BC01F801828D938D0E9439
:102E3000E7F7C80FD91F63E071E28EE091E20E94CC
:102E40003DF88C01009771F069E070E080E090E05F
:102E50000E94DBF5BC01F801828D938D0E94E7F79B
:102E6000C80FD91FCE01DF91CF911F910F91089507
:102E7000A6E7B4E2E6E0F5E280E08D9381938F5F10
:102E80008039D9F780E090E0089580E090E00895DF
:102E90008039910528F4FC01EA58FB4D808190E0CF
:102EA00008958F929F92AF92BF92CF92DF92EF924E
:102EB000FF920F931F936B017C010E94C9F590E074
:102EC000A0E0B0E0C816D906EA06FB06A0F0C701EC
:102ED000B6010E94DBF5DCDF0E9438F64B015C0195
:102EE000C701B6010E9402F695018401080F111D69
:102EF000211D311D02C097018601B801C9011F9132
:102F00000F91FF90EF90DF90CF90BF90AF909F9088
:102F10008F9008954F925F926F927F92AF92BF927F
:102F2000CF92DF92EF92FF920F931F93CF93DF9395
:102F3000CDB7DEB7D450CDBFDEBF5C018B018617A5
:102F4000970709F475C082E0A816B10408F470C0B0
:102F50006230710508F46CC0E8EFAE16EFE0BE0613
:102F600008F066C0683FFFE07F0708F061C0C50158
:102F70000E9438F62B013C01C8010E9438F66B0113
:102F80007C01B301A201CE018F5F9D4F0E949BF493
:102F9000B701A601CE0101960E949BF4B301A201E4
:102FA000CE0101960E9417F5B701A601CE018F5FF1
:102FB0009D4F0E9417F58FEF481A580A680A780A41
:102FC000B301A201CE018F5F9D4F0E949BF4EFEFF2
:102FD000CE1ADE0AEE0AFE0AB701A601CE0101965C
:102FE0000E949BF4B301A201CE0101960E9417F545
:102FF000B701A601CE018F5F9D4F0E9417F5C50155
:103000008A5F9A4DFC012081A22FB0E0AA58BB4DE7
:103010004C910A5F1A4DF8013081E32FF0E0EA5835
:10302000FB4D50815C934083FC013083F801208389
:10303000DC5FCDBFDEBFDF91CF911F910F91FF907D
:10304000EF90DF90CF90BF90AF907F906F905F90A8
:103050004F90089540E054E06FEF70E086E997E20A
:103060000F94BE0C80E090E0089580E090E0089519
:1030700080E090E0089580E090E008959C01CB010D
:10308000BA0149E0660F771F881F991F4A95D1F74B
:103090004091CF0147FDFCCF40E052E0C9010F94C1
:1030A000D30C80E092E008959C01CB01BA0159E075
:1030B000660F771F881F991F5A95D1F74091CF014E
:1030C00047FDFCCF40E052E0C9010F94EE0C80E0D8
:1030D00092E0089580E092E0E6E9FBE2DF019C01E6
:1030E0001D9221503040E1F780E090E0089580E0AB
:1030F00090E00895411551056105710529F421E01D
:1031000040E050E0BA0113CD423051056105710530
:1031100058F420E032E0E6E9FBE2DC0101900D9298
:1031200021503040D9F709C0FC0180E092E0DF0176
:103130009C011D9221503040E1F780E092E008951B
:10314000CF92DF92EF920F93CF93DF9300D0CDB762
:10315000DEB76C0121E084E691E089839A832B83BA
:10316000411551056105710599F42FEF30E048E1F3
:1031700060E070E0CB0192DC8AE1E82E01E020E023
:1031800030E0A901B601CE010196BEDD9C0113C05D
:10319000423051056105710560F480E092E0F6016E
:1031A000A6E9BBE201900D920197E1F720E032E041
:1031B00002C020E030E0C9012396CDBFDEBFDF9121
:1031C000CF910F91EF90DF90CF90089580E090E045
:1031D000089580E090E0089533CDDBCD80E090E06D
:1031E000089580E090E00895452B462B472B29F465
:1031F00022E040E050E0BA019ACCFC0180E092E08D
:10320000DF019C011D9221503040E1F780E092E007
:10321000089580E090E0089580E090E00895CF92D6
:10322000DF92EF92FF920F931F93CF93DF93EC0106
:1032300080E092E0FE019C01119221503040E1F7C4
:10324000452B462B472B09F049C08CE0E0E9F0E024
:10325000DE0101900D928A95E1F7FE01709680E003
:1032600027E038ED833089F01092C2011092C1013D
:103270008093C0012093CA0134BF9091CB0191602B
:103280009093CB019091C40190838F5F31968630EB
:1032900049F78091D0018F8B80E888A38FEF89A3B5
:1032A0008AA38DEF8BA318A619A61AA61BA60EE457
:1032B0001EEF21E03327E096B801C901005FC12C61
:1032C000D12C7601C394C60ED71EE81EF91E40E02D
:1032D00015DC8993C701B6010C11F1CF80E092E0B3
:1032E000DF91CF911F910F91FF90EF90DF90CF90E2
:1032F00008950F931F93CF93DF93CDB7DEB7EC976D
:10330000CDBFDEBF0EE311E207D3F80181938F0139
:10331000F1E206341F07C1F70E9459F090D38823C9
:1033200009F4EFC080913E2190913F21953009F43E
:1033300068C038F4913059F170F0933009F0E1C071
:1033400026C0983009F4B9C0993009F4BFC096304E
:1033500009F0D7C06AC0803821F0823809F0D1C0A6
:1033600003C010913B210EC0809142218F70F2D298
:10337000E0914821F0914921118112FB112710F9A8
:1033800080E0E8D230D3812FD6D280E09BC0882362
:1033900019F0823009F0B5C08F71823009F0B1C0E8
:1033A00080914021811129C0009142211091432137
:1033B0000F7011270115110509F4A3C0802FCAD27F
:1033C00080913F21833011F4F3D217C0E09148215E
:1033D000F091492181818B7F818384E8809FF00176
:1033E000819FF00D1124E457FE4D1082E091482199
:1033F000F091492180818E7F808380E0ABD2F3D22F
:1034000063C081117EC0109140211F77ECD20BD494
:1034100048D38823E9F31093C304112311F083E008
:1034200001C082E080933D216CC08058823008F05A
:1034300068C080914021909141218C3D23E092070A
:1034400059F583E08A838AE389834FB7F894DE01D4
:10345000139620E038E052E05093CA01E32FF0E0E9
:10346000E4911092CA0120FF03C0E295EF703F5F24
:10347000EF708E2F90E0EA3010F0C79601C0C09632
:103480008D939D932F5F2C3139F74FBFACD26AE3F8
:1034900070E0CE0101960EC0AE01455C5F4F6091B9
:1034A00042210E945EF08C01009759F19CD2B80134
:1034B0008BAD9CAD90D121D224C0803811F593D230
:1034C00080913A2138D200D2AED31BC0811119C0ED
:1034D000809140218230A8F486D28091402180934F
:1034E0003A21A1D380913A21811104C08091C30473
:1034F000882311F084E001C081E080933D210E9487
:1035000055F09DD2882311F06ED252D2EC96CDBFE9
:10351000DEBFDF91CF911F910F9108950895CF9352
:1035200080913D21882351F0C0914A2180E012D240
:1035300086D28111DEDE8C2FCF910CC2CF910895FF
:10354000DF92EF92FF920F931F93CF93DF93EC01E3
:103550008B0180D3D82E811135C00115110529F0BA
:10356000F80120813181C21BD30BE12CF12C26C044
:103570002091462130914721F901EF5BFF4F908167
:10358000F901E05CFF4F8081981790F09DD1011503
:10359000110551F0F801808191818E0D9F1D80836E
:1035A000918395E0D92E0EC055D3882339F009C0F8
:1035B00080E0C1D12197FFEFEF1AFF0A2097C1F6F3
:1035C00001C0D82E8D2DDF91CF911F910F91FF90CB
:1035D000EF90DF900895BF92CF92DF92EF92FF922B
:1035E0000F931F93CF93DF937C018B01EA0132D3BA
:1035F000B82E811138C0209731F028813981021B03
:10360000130BE20EF31EC12CD12C28C020914621B1
:1036100030914721F901EF5BFF4F9081F901E05CA8
:10362000FF4F8081981788F04FD179DF209749F0BC
:10363000888199818C0D9D1D8883998325E0B22E08
:1036400012C008D3882351F00DC0F70181917F018A
:1036500072D101501109FFEFCF1ADF0A01151105D0
:10366000A9F601C0B82E8B2DDF91CF911F910F913C
:10367000FF90EF90DF90CF90BF900895BF92CF92D0
:10368000DF92EF92FF920F931F93CF93DF936C0122
:103690008B017A01DFD2B82E81113FC0E80121975A
:1036A000CC0DDD1DE114F10439F0F70120813181E9
:1036B000021B130BC21BD30BC12CD12C29C0209190
:1036C000462130914721F901EF5BFF4F9081F901CD
:1036D000E05CFF4F8081981798F0F6D020DFE1146E
:1036E000F10451F0F701808191818C0D9D1D808343
:1036F000918335E0B32E11C0ADD2882349F00CC0C0
:10370000888119D1219701501109FFEFCF1ADF0AE3
:1037100001151105A1F601C0B82E8B2DDF91CF91B7
:103720001F910F91FF90EF90DF90CF90BF90089581
:10373000BF92CF92DF92EF92FF920F931F93CF939E
:10374000DF937C018B01EA0185D2B82E811138C04C
:10375000209731F028813981021B130BE20EF31EF2
:10376000C12CD12C28C02091462130914721F9014C
:10377000EF5BFF4F9081F901E05CFF4F808198176C
:1037800088F0BBD0CCDE209749F0888199818C0DE0
:103790009D1D8883998345E0B42E12C05BD2882397
:1037A00051F00DC0B9D0F70181937F01015011098B
:1037B000FFEFCF1ADF0A01151105A9F601C0B82ED7
:1037C0008B2DDF91CF911F910F91FF90EF90DF90A4
:1037D000CF90BF900895DF92EF92FF920F931F93C7
:1037E000CF93DF93182F092FEB0180914A21806836
:1037F000B1D020914421309145212C173D0720F074
:10380000209719F461D001C0E901E12EF02ED12CEE
:103810003FC080913D21811102C082E04DC08530C2
:1038200011F483E049C00BD1811145C021D1811130
:103830003DC037D1882361F120914A2180914621F2
:1038400090914721FC0127FF05C0EF5BFF4F0081EE
:1038500010E012C0E05CFF4F0081FC01EF5BFF4F06
:10386000808110E0081B110907C0F70181917F01D9
:1038700062D021970F5F1F4F209719F00830110574
:10388000A0F3DD24D3940830110509F0D12C1CD00D
:10389000209709F0BECFD110BCCF08C080913D2148
:1038A000882309F4BACF853009F4BBCFE1D088234F
:1038B000A9F380E001C081E0DF91CF911F910F91CA
:1038C000FF90EF90DF900895E0914821F091492119
:1038D000A0914621B0914721AF5BBF4F8C9190E002
:1038E0008283938380818D798083E0914621F0915A
:1038F0004721EF5BFF4F10820895E0914821F0913E
:10390000492180818D798083E0914621F091472182
:10391000EF5BFF4F108208958091462190914721DF
:10392000FC01EF5BFF4F2081DC01A20FB11D8C91E8
:103930002F5F208308952091462130914721F9017E
:10394000EF5BFF4F9081D901A90FB11D8C939F5F51
:103950009083089580934A21482F4F7094E8499F9F
:1039600090011124255B3E4D6091C6047091C704FF
:1039700090E1499FA001112487FF0FC02E5B3F4FAC
:103980002093462130934721CA010896860F971F3E
:1039900080934821909349210895209346213093A4
:1039A0004721460F571F40934821509349210895BE
:1039B000E0914821F0914921818184608183E091E7
:1039C0004821F09149218181807C803459F4809193
:1039D0004A218058BFDFE0914821F091492181813F
:1039E00084608183089580914A218F77B3DFE091CD
:1039F0004821F091492180818D788083E091482190
:103A0000F0914921808181608083E0914621F0918D
:103A10004721EF5BFF4F108280914A2180689ADF37
:103A2000E0914821F0914921808181608083E0917B
:103A30004621F0914721EF5BFF4F1082089580915E
:103A40004A218F7787DFE0914821F09149218081D9
:103A500084FF0CC0209146213091472182819381BF
:103A6000F901E05CFF4F808381E0089580E00895D4
:103A700080914A218F776EDFE0914821F0914921B2
:103A8000808185FF0CC020914621309147218281A1
:103A90009381F901E05CFF4F808381E0089580E02D
:103AA000089580914A21806855DFE0914821F09186
:103AB000492180818695817008951F93CF93DF936C
:103AC0001F921F92CDB7DEB7182F4A83698342DF5A
:103AD000E0914821F09149211182E0914821F09133
:103AE0004921812F881F8827881F880F8083E091B4
:103AF0004821F091492169816183E0914821F09149
:103B0000492112821382209146213091472124833A
:103B10003583110F110B4A811423F901E05CFF4F2B
:103B20001083F901EF5BFF4F108281E00F900F903F
:103B3000DF91CF911F910895CF92DF92EF92FF9284
:103B40000F931F93CF93DF931F921F92CDB7DEB7D2
:103B5000E62E6C01F12C46C0F6015081511105C0D2
:103B6000F394F5E0CF0ED11C3DC0F6010181128126
:103B700083819481923010F048E101C048E028E050
:103B800030E090E003C09F5F220F331F2017310702
:103B9000D0F3252F2F7030E02230310514F080E073
:103BA00024C001341105D8F7942B9F7E882319F087
:103BB000813029F402C0906405C0906C0CC09068FC
:103BC000811109C0402F692F852F805859839A830E
:103BD00074DF9A815981402F692F852F6EDF811103
:103BE000BFCFDDCFFE10B8CF81E00F900F90DF91F7
:103BF000CF911F910F91FF90EF90DF90CF9008959C
:103C0000E0ECF4E0A681B78119961C92A681B781F9
:103C100011961C92A681B78159961C920680F78155
:103C2000E02D118A089580913E2187FD04C039DF7F
:103C3000882351F00EC01CDF811105C080913D2109
:103C40008111F9CF089559CE80913D218111EFCF97
:103C500008953ACE1F93CF93DF93E091C604F0917D
:103C6000C704C0A1D1A114E602C0EC01122F8091BB
:103C70004A218078803851F414DF811105C0809189
:103C80003D21811105C01CC080E01FC0F1DEF5CFD1
:103C90008530C1F0E0914821F0914921818182FD78
:103CA00013C0E091C604F091C70480A191A18C17C4
:103CB0009D07E9F2212F21501111D7CF84E005C0D3
:103CC00082E003C083E001C081E0DF91CF911F91CA
:103CD0000895CF93DF93E0E4F0E014828481836061
:103CE00084834CD052D0C0ECD4E088818F77888315
:103CF00088818068888310923D2110923A21109229
:103D00003B2188818064888348E068E480E8D5DED0
:103D100048E068E480E0D1DE888580648887898116
:103D200081608983DF91CF910895CF93DF933FB76F
:103D3000F894C0ECD1E022E02A87EAE1F0E0E491D7
:103D4000A0ECB4E0DA96EC93DA97EBE1F0E0E491E2
:103D5000DB96EC93DB971A8684E592E28E7F1696CB
:103D60008D939C93179781E18C9318962C933FBF6A
:103D700081E080933C21DF91CF91ABCFE0ECF4E088
:103D800080858370808711860895E0ECF4E08FEFE2
:103D90008287848708951F920F920FB60F92112485
:103DA0000BB60F922F933F934F935F936F937F9335
:103DB0008F939F93AF93BF93EF93FF938091CA0428
:103DC00087FF08C08091C80487FF04C080E8809303
:103DD000CA04A4DB8091CA0486FF07C080E48093F4
:103DE000CA0410923D210E9454F08091CA0485FFBC
:103DF00014C080E28093CA0480913A21882311F094
:103E000084E007C08091C304882311F083E001C0DF
:103E100081E080933D210E9453F08091CA0484FF89
:103E200014C080E18093CA0482E080933D21109207
:103E30003A211092C304E4DE48E068E480E83DDE05
:103E400048E068E480E039DE69DBFF91EF91BF91E3
:103E5000AF919F918F917F916F915F914F913F9122
:103E60002F910F900BBE0F900FBE0F901F901895C3
:103E7000CF93DF93EC01E3DD882339F1888190E073
:103E8000209142213091432128173907F1F4809184
:103E90003F218E3F59F08F3FC1F480913E21813206
:103EA000A1F4A1DDC0DE81E088AF0FC080913E218A
:103EB000813A59F498DDF5DD8823E9F38B8581504B
:103EC0003ADD02DDDF91CF91AECEDF91CF91089543
:103ED000CF93DF93EC010C96FC018DE2DF011D9284
:103EE0008A95E9F782E08C83898761E0CE010196AB
:103EF00023DE882331F061E0CE010696DF91CF9179
:103F00001BCE80E0DF91CF910895EF92FF920F9347
:103F10001F93CF93DF931F921F92CDB7DEB78C0113
:103F200080913D21843009F001C1F801868112DDC4
:103F30009FDD882309F4AAC0F80186810BDD198270
:103F40001A827801FCE0EF0EF11C03C080AD8111F4
:103F50009DC0AE014F5F5F4F6FE070E0C701E8DBCF
:103F6000F801853099F384859585A685B7858535D3
:103F70009345A244B34469F4F801918D8385981761
:103F800040F4808D8F7129F4828D882311F0813166
:103F900030F00EDDF8018181DDDC0ADD77C01982A9
:103FA0001A827801FBE1EF0EF11C04C0F80180AD2C
:103FB00081116CC0F801628DAE014F5F5F4F70E000
:103FC000C701B6DB853091F398DCF801808D87FF5F
:103FD00002C08181BFDCC8010E945DF091E098279A
:103FE000F80197AB45E553E562E473E543A754A7B1
:103FF00065A776A7408951896289738947A750AB25
:1040000061AB72AB448955896689778943AB54AB00
:1040100065AB76AB811105C0452B462B472B09F0CC
:10402000C7DCF801868196DC05C079DAF80180AD3D
:1040300081112CC0E0914821F0914921818182FDBC
:10404000F4CFF801818186DC05C069DAF80180AD22
:1040500081111CC0E0914821F0914921818182FDAC
:10406000F4CF19821A827801FBE2EF0EF11C04C032
:10407000F80180AD81110AC0AE014F5F5F4F6DE066
:1040800070E0C701A8DA853099F31EDCF80180AD35
:10409000882309F44BC08681E82FEF7087FF07C0A3
:1040A00024E8E29FF0011124E253FE4D06C084E8AB
:1040B000E89FF0011124E457FE4D1082F801818140
:1040C000E82FEF7087FF07C024E8E29FF00111247A
:1040D000E253FE4D06C084E8E89FF0011124E45746
:1040E000FE4D1082F801868135DCE0914821F09187
:1040F000492181818B7F8183E0914821F091492181
:1041000080818E7F8083F801818124DCE0914821C9
:10411000F091492181818B7F8183E0914821F09149
:10412000492180818E7F8083F80110AE0F900F901F
:10413000DF91CF911F910F91FF90EF900895FB01B8
:10414000DC0102C001900D9241505040D8F7089513
:10415000DC0101C06D9341505040E0F70895FB0130
:10416000DC014150504030F08D910190801919F4DC
:104170000020B9F7881B990B0895E0ECF1E0A785C2
:10418000A7FDFDCFA485A860A4876050704FD7CF4E
:1041900003D0808199270895E0ECF1E0378537FD61
:1041A000FDCF348538603487FC01E050F04F08952E
:1041B000DC01A40FB51F4150504040F0CB01840FEB
:1041C000951F2E9105D041505040D8F70895262FC5
:1041D000E3DF0080021611F004D0019701970895E3
:1041E000262FE0ECF1E0378537FDFDCF3485377FB2
:1041F0003487378531FF09C036E3328738ED34BF65
:1042000031E03387378537FDFDCF33E33287808355
:1042100091831282248325E3228728ED31E024BF95
:10422000338701960895F894FFCF00814000000184
:10423000014000000101000000000000000000003B
:10424000000000000000000000000000000000006E
:10425000000000000000000000000000000000005E
:10426000000000FF700000000000000A00000000D5
:1042700000000000000026034100540078006D009B
:1042800065006700610031003200380041003300F2
:10429000550020006400690073006B0000002203D9
:1042A0005300740065007000680061006E0020001B
:1042B000420061006500720077006F006C006600CC
:1042C00000000403090409022000010100803209F2
:1042D000040000020806500007058102400005079F
:1042E0000501024000051201100100000008EB0367
:1042F000452001000102DC01982074204C2004229A
:1043000026008000021F00000041746D656C0000F3
:10431000004154786D656761313238413355000092
:1043200000302E3030454550524F4D202042494EEE
:10433000555345525349474E4649524D57415245B0
:10434000424F4F544C4F414450524F445349474EB3
:10435000444556494E464F20524541444D45202044
:10436000545854000000000000000000000000004D
:10437000000000000000000000000000000000003D
:10438000000000000000000000000000000000002D
:10439000000000000000000000000000000000001D
:1043A000000000000000000000000000000000000D
:1045D0000000000093C0000088C0000096C00000EA
:1045E0002FEF089577C0000020E208952FEF08957F
:1045F0009CC000002FEF08952FEF08952FEF08952E
:104600002FEF08952FEF08952FEF08952FEF0895BE
:104610002FEF0895000000000000000000000000DF
:10462000000000000000000000000000000000008A
:10463000000000000000000000000000000000007A
:10464000000000000000000000000000000000006A
:10465000000000004154786D6567613132384133A4
:1046600055206469736B202870726F746F74797051
:1046700065290032303134303432305431323435FF
:104680005A5342006279205374657068616E20420B
:10469000616572776F6C6620286D617472697873DA
:1046A000746F726D40676D782E6465292C20496C9B
:1046B0006D656E61752032303134000000000000FD
:1046C00000000000000000000000000000000000EA
:1046D000000000002FEF7D3F39F46F3F29F45F3F6A
:1046E00019F4403809F4222708952F932227F2DF86
:1046F0002F3F11F42F9109C0DF9008952F932227A7
:10470000E9DF2F3FF9F32F9100C0B0923B00F60193
:10471000B22E06D02DE9B092CA0120933400E8955C
:104720002091CF01207CE1F708950C94DCF000008B
:104730000000000000000000000000000000000079
:104740000000000000000000000000000000000069
:104750000000000000000000000000000000000059
:104760000000000000000000000000000000000049
:104770000000000000000000000000000000000039
:104780000000000000000000000000000000000029
:104790000000000000000000000000000000000019
:1047A0000000000000000000000000000000000009
:1047B00000000000000000000000000000000000F9
:1047C00000000000000000000000000000000000E9
:1047D00000000000CF93DF93CDB7DEB7D450CDBF3C
:1047E000DEBFF8948091A00680648093A00680913B
:1047F000A40680648093A4060E9426016933714355
:104800008C4E9E4161F08091A70680648093A7063C
:104810008BE792E90197F1F700C00000F4CF80E048
:1048200090E48C01012F112706959170892B11F0CE
:104830000F5F1F4FC12CD12C7601C016D10608F096
:1048400057C0B701A60140515F4F6F4F7F4FCE0158
:104850008F5F9D4F0E94CA02B701A601CE0101964B
:104860000E947F01BE016F5F7F4FCE018F5F9D4F22
:104870000E94DD012FEFC21AD20AE20AF20A892B46
:10488000E1F2C12CD12C7601B701A601CE018F5FD8
:104890009D4F0E947F01B701A60140515F4F6F4FAE
:1048A0007F4FCE018F5F9D4F0E94A5038FEFC81AE7
:1048B000D80AE80AF80AC016D10630F39FED23E9BA
:1048C00084E0915020408040E1F700C000000E9449
:1048D000DE038091A70680648093A7069FE72DE8FA
:1048E0008BE5915020408040E1F700C00000F1CFFF
:1048F0009FED23E984E0915020408040E1F700C023
:1049000000000E94DE038091A70680648093A706C2
:104910009FE728E381E0915020408040E1F700C00C
:084920000000F1CFF894FFCF75
:02492800FF008E
:00000001FF
